:020000040000FA
:1000000001288316FF2390002E30850006309500CE
:1000100000308100831200308B00073099003230AD
:10002000A200F930A0000000A00B1328A20B112899
:1000300000341930A100F930A0000000A00B1D28E9
:10004000A10B1B280034F930A0000000A00B2528CC
:10005000003411308500851A302885193628642827
:10006000851933284D28113085002B28851839280B
:100070003C2805193F284628103085002B281030D1
:1000800085000F20113085000F202B2810308500AF
:1000900019201130850019202B2885185028532845
:1000A000051956285D28013085002B280130850070
:1000B0000F20113085000F202B28013085001920DA
:1000C0001130850019202B28851867286A28051902
:1000D0006D287428003085002B28003085000F2003
:1000E000113085000F202B28003085001920113099
:0600F000850019202B28F9
:02400E00D43F9D
:00000001FF
